:10343000754A06121A1F203104E52F70F9121A6816
:10344000754A061219DF80E822754A04121A1FE530
:103450002F70FC121A68754A041219DF7F011214CA
:10346000537E007FFF8F0512322CDFF97E007FFF35
:10347000900000C007123269EFF0A3D007DFF422FA
:10348000754A01121A1FE52F70C5121A68754A0194
:103490001219DF22754B011214537808302FFDE505
:0B34A0003D2430121424C22FD8EA2271
:100E9B00758400854FD28550D37584018551D285D9
:100EAB0052D3E4F550F54F30080685534F85545017
:100EBB0030090CE54F2555F54FE5503556F55030BB
:100ECB000A10E5338534F0A4254FF54FE5F0355086
:100EDB00F550300B10E50A8537F0A4254FF54FE59B
:100EEB00F03550F550300C10E5118536F0A4254F38
:100EFB00F54FE5F03550F550E4F552F55130101043
:100F0B00855351855452E554C3953B4003853B5261
:100F1B00301116E556C3953A4003853B56E55125EE
:100F2B0055F551E5523556F552301210E5338534EF
:100F3B00F0A42551F551E5F03552F552301310E57B
:100F4B000A8537F0A42551F551E5F03552F55230AD
:100F5B001410E5118536F0A42551F551E5F0355205
:100F6B00F552301510E5188535F0A42551F551E5EE
:100F7B00F03552F552301610E5288539F0A425517D
:100F8B00F551E5F03552F552301710E5298538F05B
:100F9B00A42551F551E5F03552F552E552C3953C78
:100FAB004003853C5222901018303303120FD3307C
:070FBB003403120FE330368E
:100FC20003121007303503121006303703121017C0
:100FD20022E50B2509F50BE50C3508F50C93F50A0E
:100FE20022E512250EF512E513350DF51393C31301
:100FF200F8E5142510F514E515350FF51593C3130F
:1010020028F5112222E5192517F519E51A3516F5E5
:101012001A93F51822227F8285888C8F9295989B4D
:101022009EA1A4A7AAADB0B3B6B9BBBEC1C3C6C97F
:10103200CBCED0D3D5D7D9DCDEE0E2E4E6E7E9EBEC
:10104200EDEEF0F1F2F4F5F6F7F8F9FAFBFCFCFD3F
:10105200FDFEFEFEFEFEFEFEFEFEFEFDFDFCFCFBB8
:10106200FAFAF9F8F7F6F4F3F2F0EFEDECEAE8E762
:10107200E5E3E1DFDDDBD8D6D4D1CFCDCAC8C5C226
:10108200C0BDBAB7B4B2AFACA9A6A3A09D9A9794BB
:10109200908D8A8784817E7A7774716E6B686562BF
:1010A2005F5C595653504D4A4744423F3C393734AE
:1010B200322F2D2A282624211F1D1B19181614121F
:1010C200110F0E0C0B0A08070605040403020201A5
:1010D2000100000000000000000000010102020304
:1010E2000405060708090A0B0D0E10111315161830
:1010F2001A1C1E20222427292B2E303335383A3D44
:10110200404245484B4E515456595C606366696C87
:061112006F7275787B7F0F
:10138100D2F4C2F5C2F675840F85F0C81211B1749A
:10139100031213D01211A574031213D01211881263
:1013A100118874031213D012118874021213D0120F
:1013B1001188742812143C740612143C740E121411
:1013C1003C740112143C1211A5748012143C22C009
:1013D10000A2E092F3A2E192F2A2E292F1A2E392E0
:1013E100F0D2F475840F85F0C8C2F47830D8FE8548
:1013F100F0C87830D8FED00022C00075840FA2E476
:1014010092F3A2E592F2A2E692F1A2E792F0D2F46F
:1014110085F0C8C2F47830D8FE85F0C87830D8FE9F
:10142100D00022EF75840FD2F5C2F685F0C81213F1
:10143100FA1211881213D01211882275840FC2F585
:10144100C2F685F0C81213FA1211881213D01211C4
:101451008822EF14A2E492E6C2E4D2E712143C22FD
:10146100740F12143C22740D12143C227F011214C9
:101471005378107F20121424D8F9227F11121453AB
:1014810078107F20121424D8F9227F011214537886
:10149100207F20121424D8F922C0077F018004C0C4
:1014A100077F11121453D007C082C083C007EF75A4
:1014B100F0109014CB1211C97810E493FF12142488
:0914C100A3D8F7D007D083D08234
:1014CA002220202020202020202020202020202010
:1014DA002030313233343536373839414243444586
:1014EA00462020205253343232205445535420206F
:1014FA002020202052533233322054455354202086
:10150A002020205445535420204641494C4544202C
:10151A002020205445535420205041535345442001
:10152A00202020454550524F4D20544553542020E9
:10153A0020204155582052454C4159205445535476
:10154A002020205055534820544F2054414C4B20C2
:10155A002054455354203320434841522F53554277
:10156A00205445535420464958454420535452491F
:10157A004E544553542056415249422053545249DD
:10158A004E464143544F52592044454641554C54C6
:10159A002050524F4752414D4D494E47204D4F44DE
:1015AA004553494D504C45582052455045415445A4
:1015BA00522020205245434F5244494E4720202072
:0115CA002000
:10322C00758400D2C2C2C6D2C6C2C4D2C5C2C33013
:10323C00C3FD74A0F5C2C2C5C2C330C3FD8EC2C2E9
:10324C00C330C3FD8FC2C2C330C3FD8DC2C2C330F5
:10325C00C3FDD2C4C2C320C4FD1211A522758400C3
:10326C00C2C3D2C530C3FD74A0F5C2C2C5C2C3303F
:10327C00C3FD8EC2C2C330C3FD8FC2C2C330C3FDF7
:10328C00C2C4D2C5C2C330C3FD74A1F5C2C2C5C28B
:10329C00C330C3FDC2C2C2C330C3FD85C207D2C492
:0632AC00C2C320C4FD2294
:080003000215CB000000000013
:08000B000215CC00000000000A
:08001300021757000000000075
:08001B003200000000000000AB
:09002300320000000000000000A2
:08002B000215CF0000000000E7
:08003300320000000000000093
:0A003B003200000000000000000089
:0900430032000000000000000082
:08004B0032000000000000007B
:08005300320000000000000073
:08005B0002162E000000000057
:08006300320000000000000063
:08006B0002164C000000000029
:080073000215D5000000000099
:08007B0002175800000000000C
:0800830002162B000000000032
:08008B0032000000000000003B
:1000930002177600000000000000000000000000CE
:1000A3003275FF0775FFDE75FFAD75840F75E107C8
:1000B30075E20475E34475840F75A43575A5097558
:1000C300A6FF75A7FF759CFF759D00759E00759F24
:1000D300F075D8FF75E8FF75F80F75AD0F758401DE
:1000E30075893075888F75840275893075888F7529
:1000F300840F758A80758C67780874FF0000000090
:100103000000000000000000D5E0F1D8EDE58C30E0
:10011300E7FB759701758A0043890475840075B7F9
:100123001075840F438901758D01758F01758E02DA
:100133007480D5E0FD438902E58930E4FB759702BD
:1001430075840075D10775840075BB0175BA007598
:10015300BCF075C70075C60075C5FF75C4FF75E8AB
:100163008175840275BB0475BA0075BCF175C60050
:1001730075C4FF75E88875840075D484758401752A
:10018300D484758400C2F8759A47759D1A43F8099B
:1001930075870075840075B90075A90075910075A0
:1001A300985075840175981075840075C04075C3A7
:1001B3000075CFC9758400758E0075892075880513
:1001C300758400758A00758B6F758CF4758D6F431C
:1001D300885075840075C90075CA0075CB0075CC4D
:1001E3000075CD0075C80075840175C91875CA807E
:1001F30075CBFB75CDFB75CC80D2CA75840275C9EE
:100203001875CA1275CBF775CDF775CC12D2CA75AE
:10021300840075EF0075A8AF75B80075E6A475E79F
:100223001775F60075F7019000007F007E20E4F05B
:03023300A3DFFC4A
:10023600DEFA7534FF7535FF7536FF7537FF75388D
:10024600FF7539FF753AFF753BFF753CFF751D0A53
:07025600751E0A751F062248
:1015CB0032C28D32758400C2CF32C0E0C083C0827C
:1015DB00C0D0C000C0F0C2CFB239203923120E9B4D
:1015EB00151BE51B7009751B0A7584017588AF15F2
:1015FB001CE51C7009751C607584027588AF800E24
:10160B00120FB1152AE52A7005752A04D28B758441
:10161B0000D2ECD0F0D000D0D0D082D083D0E0324A
:10162B00C2CF32C0E0C0D0E52B6002152BE52E6097
:10163B0002152EE55C6002155C75888FD0D0D0E06A
:10164B0032C0E0C0D0C08420301375840F30DF254A
:10165B00E5E8540FF53DD230753EC88018153EE5D0
:10166B003E7006E53DD2E7F53D75840F20DF06C2DF
:10167B0030D22FD22B20321475840F30F828E5E8A6
:10168B0054F0C4F53FD2327540C8801A1540E5407E
:10169B007006E53FD2E7F53F75840F20F808C2329C
:1016AB00D231D22AD21CE52C6002152CE5596002EE
:1016BB001559E55B6002155BE55D6002155DE56341
:1016CB0060021563B2A1151DE51D7077751D0AE546
:1016DB002D6002152DE52F6002152FE55E600215BA
:1016EB005EE55F6002155FE55760021557E55860D0
:0D16FB00021558B2A0E54C6002154CE54DFB
:101708006002154DE54E6002154EE56160021561F7
:10171800E57060021570151EE51E702A751E0AE533
:101728005A6002155AE56260021562E57160021599
:1017380071E57260021572151FE51F7009751F06A5
:10174800E56060021560D084C28DD0D0D0E032321E
:10175800202E0DD22E85BF5685BE5575BB01800B38
:10176800C22E85BF5485BE5375BB00C2ED32C0E0A2
:10177800C0D0E541B4000A054185BE3375BB07807A
:101788003DB4010A054185BE3075BB048030B40202
:101798000A054185BE3375BB068023B4030A05419B
:1017A80085BE3175BB048016B4040A054185BE3375
:1017B80075BB05800975410085BE3275BB04C2ED55
:0517C800D0D0D0E0329A
:1011180075840FD2FD2275840FC2FD2275840FD20B
:10112800FC2275840FC2FC2275840FD2FED21E22C7
:1011380075840FC21EC2FE22C29322D293227584E6
:101148000FA2FA2275840FA2F92275840FA2DD225C
:1011580075840FA2DE22A2922275840FA2DA22756C
:10116800840FA2DB2275840FA2D82275840FA2D91E
:101178002200000000000000000000000000002223
:10118800C000C001790478B4D8FED9FAD001D000E3
:1011980022C0007814121188D8FBD00022C0E07554
:1011A8002B05E52B70FCD0E022C0E0752B0FE52B5A
:1011B80070FCD0E022C0E0752B64E52B70FCD0E019
:1011C80022A42582F582E58335F0F58322B40A004E
:1011D80022C0E0C3997001D3D0E022B506012250A5
:1011E80007B5070122400122D322EF75F064842459
:1011F80030900063F0E5F0A375F00A842430F0A382
:10120800E5F02430F022EF75F06484243090006318
:07121800F0E5F0A375F00AF8
:10121F00842430F0A3E5F02430F0900063E0B43084
:10122F000B7420F0A3E0B430037420F02290000E72
:10123F00E0540FFFA3E0B420028019540FCF75F0D4
:10124F000AA42FFFA3E0B420028009540FCF75F03A
:10125F000AA42FFF22C006C005C00490000EE05460
:10126F000FFFFEA3E0B42003C3802C540FFDCF75F6
:10127F00F00AA42FFFA3E0B42003C3801A540FFC7D
:10128F00EE75F064A420D20EFEED75F00AA42E4088
:10129F00052C40028001D3D004D005D0062275F072
:1012AF006484F6E5F00875F00A84F608A6F00822C3
:1012BF00C0017900E6B4FF028027F908E6B4FF0306
:1012CF00C38022E975F00AA426F908E6B4FF03C328
:1012DF008013E975F00AA420D207C3264003F980D2
:1012EF0004D3D00122E9D00122E675F00AA4082622
:1012FF00227844EE1212AD75420075430078469085
:04130F0013597908ED
:10131300EF134007A3A3A3A3A3801CC0E0C000C096
:1013230001C37905E49336D4A2E4540FF6A318D984
:10133300F3D001D000D0E0D9D8E542600C75430961
:1013430075440975450975460985434285444385B6
:1013530045448546452206050200000201050000BA
:101363000402000100080400020006090004000250
:0E13730009010800040803060108060702032A
:10025D0044313233343536373839302A234142432D
:10026D0044AAA3C1C2C3C4D7ABA8A92A2341424300
:10027D000101010101010101010000000000000068
:10028D000000000000000000000000000000000061
:10029D000000000000000000000000000000000051
:1002AD000000000000000000000000000000000041
:1002BD000000000000000000000000000000000031
:1002CD00000000000000000000000101010101011B
:1002DD00010101000000000000000000000000000E
:1002ED000000000000000000000000000000000001
:1002FD0000000000000000000000000000000000F1
:10030D0000000000000000000000000000000000E0
:10031D0000000000000000000000000000000000D0
:10032D0000000000010101010101010101000000B7
:10033D0000000000000000000000000000000000B0
:10034D0000000000000000000000000000000000A0
:10035D000000000000000000000000000000000090
:10036D000000000000000000000000000000000080
:10037D0000000000000000000000000000006E06FC
:10038D0000110206190101BE10061103011501012C
:10039D0064011611040515010100000000000000A4
:1003AD000000000000000000000000000000000040
:1003BD000000000000000000000000000000000030
:1003CD000000000000000000000000000000000020
:1003DD000000000000000000010101010101010108
:1003ED0001000000000000000000000000000000FF
:1003FD0000000000000000000000000000000000F0
:10040D0000000000000000000000000000000000DF
:10041D0000000000000000000000000000000000CF
:10042D0000000000000000000000000000000000BF
:10043D0000000101010101010101010000000000A6
:10044D00000000000000000000000000000000009F
:10045D00000000000000000000000000000000008F
:10046D00000000000000000000000000000000007F
:10047D00000000000000000000000000000000006F
:10048D0000000000000000000000000020202020DF
:10049D00202020202020202020202020202020204F
:1004AD00202020202020202020202020202020203F
:1004BD00202020202020202020202020202020202F
:1004CD00202020202020202020202020202020201F
:1004DD00202020202020202020202020202020200F
:1004ED0020202020202020202020202020202020FF
:1004FD0020202020202020202020202020202020EF
:10050D0020202020202020202020202020202020DE
:10051D0020202020202020202020202020202020CE
:10052D00202020202020202020202020202020419D
:10053D004E49204E554D424552202020202020204E
:10054D00414E49204E414D452020202020415558F7
:10055D002052454C41592056414C494420202020E1
:10056D002020202020202020313D454E20202020FD
:10057D00202020202020202020414E4920202020F6
:10058D00202020202020202020202020202020205E
:10059D00202020202020202020202020202020204E
:1005AD00474C4F42414C20202020202020435443D3
:1005BD00535320434F4445202020202020204443E6
:1005CD005320434F44452020202020204C545220BE
:1005DD0052455045415445522020202020414E493E
:1005ED0020504152414D455445525320535045459D
:1005FD00442043414C4C494E472020202050544329
:10060D00204E554D424552202020202020564F4946
:10061D004345204D455353414745532020564F499F
:10062D00434520504C41594241434B202020494ED7
:10063D0056414C49442054595045202020204F55B7
:10064D0054204F462052414E4745202020494C4CC6
:10065D004547414C2056414C554520204D5553544E
:10066D002046494C4C204649454C44202020494CBD
:10067D004C4547414C20434F444520202044415494
:10068D004120414343455054454420204C494E455B
:10069D00204E554D4245523A20202020555345526B
:1006AD002050524F4752414D4D494E47555345529B
:1006BD002049443A2020202020202020564F494315
:1006CD0045205245434F5244494E472020494C4CFA
:1006DD004547414C20454E545259202020494C4C01
:1006ED004547414C2047414E4720202020202043A4
:1006FD004F4D504C45544544202020203633303644
:10070D003730363934373139373434373730373984
:10071D00373832353835343838353931353934386C
:10072D003937343130303130333130373131303198
:10073D003134313138313233313237313331313384
:10074D003631343131343631353131353631353963
:10075D003136323136353136373137313137333154
:10076D003737313739313833313836313839313926
:10077D003231393631393932303332303632313037
:10078D00323138323235323239323333323431322A
:10079D003530323534303036303037303135303128
:1007AD00373032313032333032353032363033311A
:1007BD003033323033363034333034373035303007
:1007CD0035313035333035343036353037313037EB
:1007DD0032303733303734313134313135313136E0
:1007ED0031323231323531333131333231333431DB
:1007FD0034313134333134353135323135353135BC
:10080D0036313632313635313732313734323035A3
:10081D0032313232313432323332323532323632A3
:10082D003433323434323435323436323531323584
:10083D00323235353236313236333236353236366E
:10084D00323731323734333036333131333135336A
:10085D003235333331333332333433333436333556
:10086D003133353633363433363533373134313140
:10087D00343132343133343233343331343332343E
:10088D003435343436343532343534343535343614
:10089D003234363434363534363635303335303609
:1008AD0035313635323335323635333235343635FA
:1008BD0036353630363631323632343632373633E7
:1008CD0031363332363534363632363634373033D8
:1008DD0037313237323337333137333237333437C9
:1008ED0034333735344142434445464748494A4BF2
:1008FD004C4D4E4F505152535455565758595A61AD
:10090D0062636465666768696A6B6C6D6E6F707142
:10091D0072737475767778797A303132333435363F
:10092D00373839607E21402324255E262A28295F09
:10093D002D2B3D7B7D5B5D7C3A3B3C3E2C2E3F2F32
:10094D0020202020202020202064010011021115DC
:10095D000101640200110311150101640400110469
:10096D001115010164080011051115010178060129
:10097D001106011901018202071107121500638288
:10098D0002081108121500638202091109131500DE
:10099D006382030A110A151500FF82030B110B1553
:1009AD001500FF641000110C1115051982020C11B0
:1009BD000D1415016382020D110E141500638202D0
:1009CD000E110F1415006382020F11101315016320
:1009DD00202020202020202020202020202020200A
:1009ED0020202020202020202020202020202020FA
:1009FD002054454C434F2050524F4752414D2020DB
:100A0D0020524144494F2050524F4752414D2020D2
:100A1D002050484F4E452050524F4752414D2020B7
:100A2D0020434F4D50552050524F4752414D20209D
:100A3D00202041434345535320434F44452020201C
:100A4D00205455524E204F4E2044454C41592020A4
:100A5D00205455524E204F46462044454C41592076
:100A6D005455524E2041524F554E4420444C59201E
:100A7D0044544D462054454C434F204C4556454C0F
:100A8D0044544D4620524144494F204C4556454C07
:100A9D0041555820524C5920494E56414C494420FD
:100AAD0020494E56414C49442054494D4552202031
:100ABD00202056414C49442054494D455220202078
:100ACD002020444953504C41592054494D45202034
:100ADD00204348415241435445522054494D4520ED
:100AED00202020202020202020202020313D454E78
:100AFD0020202020202020202020203130204D5368
:100B0D0020202020202020202020313030204D5347
:100B1D00202020202020202020202020205345434D
:100B2D002020202020202020202020524154494FD9
:100B3D000F3132333435360A6314FF320505050A99
:100B4D000000000000000000000000000000000098
:100B5D000000000020202020202020202020202008
:0B0B6D0020202020202020202020003D
:1045B900756064E4900000F030200B301F24124233
:1045C9005D1217CD80F530210B301F1612429C1257
:1045D90017CD80F530220B301F08121B5E1217CD44
:0345E90080F52238
:1017CD00E5607012900000E0D394004009C220C281
:1017DD0021C222C21F22900000E0122E8D18E400BB
:1017ED0018E70118EA0218ED0318F00418F20518AD
:1017FD00F40618F60718F90818FC0A18FF0B190259
:10180D000F190510190814190B15190E1919111A9C
:10181D0019141B19171E191A1F191D231920241904
:10182D00232819262919292D192C2E192F2F193254
:10183D0030193532193833193A34193D3519406498
:10184D00194365194666194967194C6E194E6F197A
:10185D00507019927119527819547919567A199242
:10186D007B195882195A83195C84195E8519618C0C
:10187D0019648D19668E19688F196B96196E9719E3
:10188D0070981972991975A01978A1197BA2197DF3
:10189D00A31980AA1982AB1985AC1987AD198AB421
:1018AD00198DB51990B61992B71994BE1997BF191C
:1018BD009AC0199DC11992C219A3F019A6F119A9BF
:1018CD00F219ACFA19AFFB19B2FC19B5FD19B8FE36
:1018DD0019BBFF000019BE0249DC0248E002419E1F
:1018ED000247BF800480028000023FFE021CCC0232
:1018FD0044E50220F1023C6B02223F023CC402236C
:10190D008D0241DF0239680228C5023DCB0224DB7E
:10191D00023E20022629023E71022777024711025C
:10192D00440502415C124048023BB780000236ED8F
:10193D00024119023EC20240910244AF023C1180A5
:10194D00468032804B8040802280458007802680F3
:10195D003F023FB2022EB3801C8035023F1302338B
:10196D00378008802B02421E02303302367E8020E3
:10197D00022F7380120234AB8016021F980233B40B
:10198D000237C8800B800C023524023F6302318F71
:10199D00024319023D750247E60238310249FA0247
:1019AD003D1D024A8D024A8E024A8F02375B024A62
:0719BD0090E4900000F0220D
:0F49DC00E4900002F0756064900000E004F022A7
:1048E00012146D12147C7BFF7A0679A91246257F7B
:0F48F00011121453C226C223900000E004F022DC
:10419E0030233D900001E0FFC223BF2A07900000AC
:1041AE00E004F022EF642370277F23121424900082
:1041BE0002E004F0E0C394034010C220C221C222E8
:1041CE00C21FE4900000F00248C09000007402F09C
:0141DE0022BE
:1047BF007BFF7A0679A912462512147C7F111214F9
:1047CF0053124A23E490003DF07F2A121424C2268C
:0747DF00900000E004F0224D
:103FFE00302346900001E0F56BC223E56B642A6026
:10400E0038AF6B1249EB5022AF6B12142490003D67
:10401E00E02404F582E43400F583E56BF090003D76
:10402E00E004F0900000E004F0227BFF7A0679D9DC
:09403E0012462590000074FAF00E
:014047002256
:101CCC00202303021E36900001E0FFC223BF2A0727
:101CDC009000007403F022EF64236003021E2712AD
:101CEC001424900005E064397077A3E064397071B6
:101CFC00A3E06439706BD228900004E0FFB4310883
:101D0C00E4900037F0021D96EFB43208E4900038EE
:101D1C00F0021DA9EFB43302803E900004E0FFB442
:101D2C003408E4900039F0021DD7EFB43508E49084
:101D3C00003AF0021DEDEFB43608E490003BF002DF
:101D4C001E03EFB437028010900004E0B438028018
:101D5C0007900004E0B4390B7BFF7A0679E9021E88
:101D6C002DC228900004E0FFB43016A3E0B430116B
:101D7C00A3E0B4300CA3E0B43007900000740AF078
:101D8C0022EFB4310C123B5A5007900000740FF044
:101D9C0022900004E0B4320C123AFA500790000082
:101DAC007414F022900004E0B43311A3E0B4300CAE
:101DBC0012489F50079000007419F022900004E024
:101DCC00B4340FA3E0B4300A124978900000741EAA
:101DDC00F022900004E0B4350FA3E0B4300A1249AD
:101DEC008D9000007423F022900004E0B4360FA311
:101DFC00E0B4300A1249A29000007428F02290003E
:101E0C0004E0B43716A3E0B43011A3E0B4300CA353
:101E1C00E0B43007900000742DF0227BFF7A067935
:0A1E2C00D912462590000074FAF068
:011E36002289
:1044E50090003C740BF090003D7407F0E490004E92
:1044F500F0A3F0900050F0900051F0A3F07BFF7A0C
:104505000579A91246251246507F1E1214539000B4
:05451500007432F022E9
:1020F100123599D3900069E09410900068E0940043
:10210100400A12461F90000074FAF022900068E025
:10211100FEA3E0FF90095675F009122E81EE75F0CD
:1021210009A42583F583E493900045F09009577540
:10213100F009EF122E81EE75F009A42583F583E4F1
:1021410093900046F0900068A3E090095875F0095B
:10215100122E81EE75F009A42583F583E493900096
:1021610047F090095975F009EF122E81EE75F009CB
:10217100A42583F583E493900048F0900068A3E0E0
:1021810090095A75F009122E81EE75F009A4258384
:10219100F583E493FD900049F090095B75F009EF38
:1021A100122E81EE75F009A42583F583E493900046
:1021B1004AF0900068A3E090095C75F009122E8145
:1021C100EE75F009A42583F583E49390004BF0901C
:1021D100095D75F009EF122E81EE75F009A42583D2
:1021E100F583E49390004CF0900068A3E090095EC1
:1021F10075F009122E81EE75F009A42583F583E4AB
:102201009390004DF0ED6015900049E075F010A439
:1022110024DDF9740935F0FA7BFF12462590004A56
:10222100E0FF601175F010A424DDF9740935F0FAAE
:0E2231007BFF124656900045E0900000F02220
:103C6B0090003C7410F090003D7407F0E490004E0F
:103C7B00F0A3F0900050F0900037E0FF900051E47B
:103C8B00F0A3EFF07BFF7A0579B912462512465067
:103C9B007F0D121453900005E0FF121424900006C0
:103CAB00E0FF121424900007E0FF1214247F1E1271
:093CBB0014539000007432F02251
:10223F00123599D3900069E09400900068E0940003
:10224F00400A12461F90000074FAF022900068E0D6
:10225F00FEA3E0FF90027D75F009122E81EE75F05E
:10226F0009A42583F583E493900045F090027E75D1
:10227F00F009EF122E81EE75F009A42583F583E4A2
:10228F0093900046F0900068A3E090027F75F009EC
:10229F00122E81EE75F009A42583F583E493900047
:1022AF0047F090028075F009EF122E81EE75F0095C
:1022BF00A42583F583E493900048F0900068A3E091
:1022CF0090028175F009122E81EE75F009A4258315
:1022DF00F583E493FD900049F090028275F009EFC9
:1022EF00122E81EE75F009A42583F583E4939000F7
:1022FF004AF0900068A3E090028375F009122E81D6
:10230F00EE75F009A42583F583E49390004BF090CC
:10231F00028475F009EF122E81EE75F009A4258362
:10232F00F583E49390004CF0900068A3E090028551
:10233F0075F009122E81EE75F009A42583F583E45B
:10234F009390004DF0ED6015900049E075F010A4EA
:10235F002499F9740435F0FA7BFF12462590004A50
:10236F00E0FF601175F010A42499F9740435F0FAA8
:0E237F007BFF124656900045E0900000F022D1
:103CC40090003C7415F090003D7407F0E490004EB1
:103CD400F0A3F0900050F0900038E0FF900051E421
:103CE400F0A3EFF07BFF7A0579C9124625124650FE
:103CF4007F0C121453900005E0FF12142490000668
:103D0400E0FF121424900007E0FF1214247F1E1217
:093D140014539000007432F022F7
:10238D00123599D3900069E09400900068E09400B4
:10239D00400A12461F90000074FAF022900068E087
:1023AD00FEA3E0FF9002D775F009122E81EE75F0B5
:1023BD0009A42583F583E493900045F09002D87528
:1023CD00F009EF122E81EE75F009A42583F583E453
:1023DD0093900046F0900068A3E09002D975F00943
:1023ED00122E81EE75F009A42583F583E4939000F8
:1023FD0047F09002DA75F009EF122E81EE75F009B3
:10240D00A42583F583E493900048F0900068A3E041
:10241D009002DB75F009122E81EE75F009A425836B
:10242D00F583E493FD900049F09002DC75F009EF1F
:10243D00122E81EE75F009A42583F583E4939000A7
:10244D004AF0900068A3E09002DD75F009122E812C
:10245D00EE75F009A42583F583E49390004BF0907D
:10246D0002DE75F009EF122E81EE75F009A42583B9
:10247D00F583E49390004CF0900068A3E09002DFA8
:10248D0075F009122E81EE75F009A42583F583E40C
:10249D009390004DF0ED6015900049E075F010A49B
:1024AD0024B9F9740435F0FA7BFF12462590004AE1
:1024BD00E0FF601175F010A424B9F9740435F0FA39
:0E24CD007BFF124656900045E0900000F02282
:1041DF007BFF7A0579D91246257BFF7A0679B912CA
:1041EF0046567F0E121453900006E0FF12142490CF
:1041FF000007E0FF1214247F1A12145390003C742E
:0F420F001AF090003D7404F09000007432F02219
:103968003029079000007403F0221246507F1E127F
:10397800145312390190006AE0FEA3E0FFD39400CB
:10398800EE94004037EF94FBEE9400502F90003CEB
:10399800741BF090003D7407F0E490004EF0A3F023
:1039A800900050F0900036E024FFFEE434FF9000D1
:1039B80051F0A3CEF09000007432F02212461F900E
:0639C800000074FAF02279
:1028C500D3900069E09400900068E09400400A12FB
:1028D500461F90000074FAF022900068E0FEA3E025
:1028E500FF90033175F009122E81EE75F009A425CC
:1028F50083F583E493900045F090033275F009EF7A
:10290500122E81EE75F009A42583F583E4939000DA
:1029150046F0900068A3E090033375F009122E810C
:10292500EE75F009A42583F583E493900047F090B4
:10293500033475F009EF122E81EE75F009A4258395
:10294500F583E493900048F0900068A3E090033588
:1029550075F009122E81EE75F009A42583F583E43F
:1029650093FD900049F090033675F009EF122E8122
:10297500EE75F009A42583F583E49390004AF09061
:102985000068A3E090033775F009122E81EE75F00B
:1029950009A42583F583E49390004BF090033875E3
:1029A500F009EF122E81EE75F009A42583F583E475
:1029B5009390004CF0900068A3E090033975F009FE
:1029C500122E81EE75F009A42583F583E49390001A
:1029D5004DF0ED6015900049E075F010A424D9F98B
:1029E500740435F0FA7BFF12462590004AE0FF603B
:1029F5001175F010A424D9F9740435F0FA7BFF128F
:0B2A05004656900045E0900000F022D3
:103DCB0090003C741FF090003D7407F090004EE49F
:103DDB00F0A37464F09000507417F0900039E0FF7A
:103DEB00900051E4F0A3EFF07BFF7A0579E91246DE
:103DFB00251246507F0F121453900006E0FF121449
:103E0B0024900007E0FF1214247F1E12145390001D
:053E1B00007432F022EA
:1024DB00123599D3900069E09403900068E0940062
:1024EB00400A12461F90000074FAF022900068E038
:1024FB00FEA3E0FF90038B75F009122E81EE75F0B1
:10250B0009A42583F583E493900045F090038C7523
:10251B00F009EF122E81EE75F009A42583F583E403
:10252B0093900046F0900068A3E090038D75F0093E
:10253B00122E81EE75F009A42583F583E4939000A8
:10254B0047F090038E75F009EF122E81EE75F009AE
:10255B00A42583F583E493900048F0900068A3E0F2
:10256B0090038F75F009122E81EE75F009A4258367
:10257B00F583E493FD900049F090039075F009EF1B
:10258B00122E81EE75F009A42583F583E493900058
:10259B004AF0900068A3E090039175F009122E8128
:1025AB00EE75F009A42583F583E49390004BF0902E
:1025BB00039275F009EF122E81EE75F009A42583B5
:1025CB00F583E49390004CF0900068A3E0900393A4
:1025DB0075F009122E81EE75F009A42583F583E4BD
:1025EB009390004DF0ED6015900049E075F010A44C
:1025FB002419F9740535F0FA7BFF12462590004A31
:10260B00E0FF601175F010A42419F9740535F0FA88
:0E261B007BFF124656900045E0900000F02232
:103E200090003C7424F090003D7407F0E490004E44
:103E3000F0A3F0900050F090003AE0FF900051E4C1
:103E4000F0A3EFF07BFF7A0579F912462512465070
:103E50007F0F121453900006E0FF12142490000705
:103E6000E0FF1214247F1E1214539000007432F0ED
:013E7000222F
:10262900123599D3900069E09400900068E0940015
:10263900400A12461F90000074FAF022900068E0E8
:10264900FEA3E0FF9003E575F009122E81EE75F007
:1026590009A42583F583E493900045F09003E6757A
:10266900F009EF122E81EE75F009A42583F583E4B4
:1026790093900046F0900068A3E09003E775F00995
:10268900122E81EE75F009A42583F583E493900059
:1026990047F09003E875F009EF122E81EE75F00905
:1026A900A42583F583E493900048F0900068A3E0A3
:1026B9009003E975F009122E81EE75F009A42583BE
:1026C900F583E493FD900049F09003EA75F009EF72
:1026D900122E81EE75F009A42583F583E493900009
:1026E9004AF0900068A3E09003EB75F009122E817F
:1026F900EE75F009A42583F583E49390004BF090DF
:1027090003EC75F009EF122E81EE75F009A425830B
:10271900F583E49390004CF0900068A3E09003EDFA
:1027290075F009122E81EE75F009A42583F583E46D
:102739009390004DF0ED6015900049E075F010A4FC
:1027490024F9F9740435F0FA7BFF12462590004A02
:10275900E0FF601175F010A424F9F9740435F0FA5A
:0E2769007BFF124656900045E0900000F022E3
:103E710090003C7429F090003D7407F0E490004EEE
:103E8100F0A3F0900050F090003BE0FF900051E46F
:103E9100F0A3EFF07BFF7A0679091246251246500E
:103EA1007F0D121453900006E0FF121424900007B6
:103EB100E0FF1214247F1E1214539000007432F09C
:013EC10022DE
:10277700123599D3900069E09400900068E09400C6
:10278700400A12461F90000074FAF022900068E099
:10279700FEA3E0FF90043F75F009122E81EE75F05D
:1027A70009A42583F583E493900045F090044075D0
:1027B700F009EF122E81EE75F009A42583F583E465
:1027C70093900046F0900068A3E090044175F009EB
:1027D700122E81EE75F009A42583F583E49390000A
:1027E70047F090044275F009EF122E81EE75F0095B
:1027F700A42583F583E493900048F0900068A3E054
:1028070090044375F009122E81EE75F009A4258313
:10281700F583E493FD900049F090044475F009EFC7
:10282700122E81EE75F009A42583F583E4939000B9
:102837004AF0900068A3E090044575F009122E81D4
:10284700EE75F009A42583F583E49390004BF0908F
:10285700044675F009EF122E81EE75F009A4258361
:10286700F583E49390004CF0900068A3E090044750
:1028770075F009122E81EE75F009A42583F583E41E
:102887009390004DF0ED6015900049E075F010A4AD
:102897002489F9740535F0FA7BFF12462590004A22
:1028A700E0FF601175F010A42489F9740535F0FA7A
:0E28B7007BFF124656900045E0900000F02294
:104711003022079000007401F02290003C742EF0CA
:1047210090003D7407F07BFF7A0679191246251235
:0E47310046507F1E1214539000007432F02286
:10440500302907900000742FF02290000BE06438EB
:104415006005A3E0B4390A12461F90000074FAF053
:10442500227BFF7A0679C912462590000BE0540FCE
:09443500F54A9000007430F022F9
:10415C0090000BE064386005A3E0B4390A12461FE6
:10416C0090000074FAF0227BFF7A0679291246251A
:10417C0090000BE0540FF54AD20AD2127534FF129C
:10418C0019C47BFF7A0679F912462590000074FE5B
:02419C00F0220F
:1040480090000BE0540FF54A302002D2081219D61E
:10405800302019203104E52F70F91219CD7BFF7A31
:104068000679F912462590000074FEF030211920D7
:104078002F04E52F70F91219CD7BFF7A0679F91212
:09408800462590000074FEF022B0
:103BB700302356900001E0FF900035F0C223121425
:103BC70024900035E0FF1249EB5021900035E0FFCB
:103BD70090003DE02404F582E43400F583EFF09093
:103BE700003DE004F0900000E004F022900035E092
:103BF700B42A079000007403F0227BFF7A0679D974
:0A3C070012462590000074FAF02226
:1036ED0030236A900001E0FF900035F0C2231214E0
:1036FD0024900035E0FFB42A0B90003CE0900000D0
:10370D00F0D22922EFB4230B90003CE0900000F0A2
:10371D00C22922900035E0FF1249EB50219000356F
:10372D00E0FF90003DE02404F582E43400F583EFE2
:10373D00F090003DE004F0900000E004F0227BFFEB
:0E374D007A0679D912462590000074FAF0220F
:1041190030233F900001E0FF900035F0121424C2D3
:1041290023900035E0FFB42A0B90003CE09000009A
:10413900F0D22922EFB4230B90003CE0900000F06C
:10414900C229227BFF7A0679D9124625900000748C
:03415900FAF02257
:0A3EC200900048E0FF70033029383B
:103ECC0012145312476C1232698F6B900046E052F9
:103EDC006BE56B60047F3180027F30121424302933
:103EEC0017C229E56B2430900024F0900034740143
:083EFC00F090000074F0F022C8
:0F3F040090004BE0FF121453900000E004F022F5
:10409100302340900001E0FF900035F0C22312145C
:1040A10024900035E0FFB42A079000007403F02249
:1040B1001249EB500F900035E090000EF090000097
:1040C100E004F0227BFF7A0679D9124625900000A0
:0440D10074FAF0226B
:1044AF00302332900001E0FF900035F0C223BF2A85
:1044BF00079000007403F022900035E0B4230790BA
:1044CF000000E004F0227BFF7A0679D9124625908E
:0644DF00000074FAF02257
:103C110012476C90006CEEF0A3EFF01232698F6BDB
:103C210090003E7401F090000EE0B431089000461F
:103C3100E0426B800E90000EE0B4301E900046E032
:103C4100F4526B90006CE0FEA3E0FFAD6B12322CDE
:103C51001249B790000074FEF0227BFF7A0679D9F1
:093C610012462590000074FAF0EF
:013C6A002237
:10352400900048E0FF700330295612145312476C80
:1035340090006CEEF0A3EFF0E4F56B900046E0FF32
:10354400E56BC39F502790006CE475F001122E6B5D
:10355400AFF0FE1232698F6C7424256BF582E4346B
:1035640000F583E56CF0121424056B80CE3029102D
:10357400C229E56B04900034F090000074F0F0224E
:1035840090003D740AF090004BE0FF121453900039
:0435940000E004F05F
:013598002210
:1034AB00302375900001E0FF900035F0C223121419
:1034BB0024900035E0FFB42A079000007403F0223B
:1034CB00EFB42308900000E004F080391249EB5070
:1034DB0038900035E0FF90003DE0FE04F074042EC0
:1034EB00F582E43400F583EFF0900046E02409FF09
:1034FB00E433FE90003DE0D39FEE6480F874809837
:10350B004016900000E004F0227BFF7A0679D91276
:09351B00462590000074FAF0222C
:10431900302337900001E0FF900035F0C2231214DA
:1043290024900035E0FFB42A079000007403F022BE
:10433900EFB42307900000E004F0227BFF7A0679AE
:0B434900D912462590000074FAF02203
:103D750012476C90006CEEF0A3EFF090003D740AD2
:103D8500F0E4F56B900046E0FFE56BC39F5027908C
:103D9500006CE475F001122E6BAFF0FE90003DE073
:103DA500FD04F074042DF582E43400F583E0FD1282
:103DB500322C056B80CE7BFF7A0679F91246259069
:053DC500000074FEF097
:013DCA0022D6
:10367E0030236B900001E0FF900035F0C22312144E
:10368E0024900035E0FFB42A079000007403F02266
:10369E001249EB501A900035E0FF90003DE0FE0419
:1036AE00F074042EF582E43400F583EFF080107B85
:1036BE00FF7A0679D912462590000074FAF022900E
:1036CE000046E02409FFE433FE90003DE0D39FEE78
:0F36DE006480F87480984006900000E004F022A9
:102EB300900048E0FF7006202903022F5E1214538E
:102EC30012476C90006CEEF0A3EFF012326912120D
:102ED3000E900046E0B40110900065E0FF12142448
:102EE300900065E0900024F0900046E0B40220904A
:102EF3000064E0FF121424900065E0FF1214249094
:102F03000064E0900024F0900065E0900025F090CC
:102F13000046E064037030900063E0FF12142490D5
:102F23000064E0FF121424900065E0FF1214249063
:102F33000063E0900024F0900064E0900025F0909E
:102F43000065E0900026F0302911C229900046E088
:102F5300900034F090000074F0F02290004BE0FFFA
:102F630012145390003D740AF0900000E004F02224
:103FB2001212645002803B12123C8F6B90004CE054
:103FC200FFE56BC39F402B90004DE0FFE56BD39F55
:103FD200502012476C90006CEEF0A3EFF0AD6B1224
:103FE200322C7BFF7A0679F912462590000074FE86
:0B3FF200F02212461F90000074FAF04D
:013FFD0022A1
:103F13001212645002803F12123C8F6B90004CE0EF
:103F2300FFE56BC39F400B90004DE0FFE56BD39F14
:103F33004004E56B702012476C90006CEEF0A3EF29
:103F4300F0AD6B12322C7BFF7A0679F9124625907D
:0F3F5300000074FEF02212461F90000074FAF076
:013F6200223C
:10333700900048E0FF700330295E12145312476C67
:1033470090006CEEF0A3EFF01232698F6B1232B27D
:10335700E4F56B7463256BF582E43400F583E0FFD5
:103367007424256BF582E43400F583EFF07463254C
:103377006BF582E43400F583E0FF121424056BE556
:103387006BC3940440CD30290FC2299000347403D5
:10339700F090000074F0F02290004BE0FF121453FD
:0C33A70090003D740AF0900000E004F07B
:0133B30022F7
:10421E007F0A122B188F6BE56B601212476C9000A1
:10422E006CEEF0A3EFF0E56B14FD12322CE56B7B18
:10423E00FF600E7A0679F912462590000074FEF0A2
:0E424E00227A06797912462590000074FAF063
:01425C00223F
:10303300900048E0FF70062029030230CE1214539B
:1030430012476C90006CEEF0A3EFF012326912128B
:103053000E90006CE475F001122E6BAFF0FE12328D
:10306300691211F2900064E0FF900024F0A3F012C3
:103073001424900065E0FF12142490006CE475F0B2
:1030830001122E6BAFF0FE1232691211F29000633F
:10309300E0FF900026F0900064E0900027F090009D
:1030A30065E0900028F0121424900064E0FF1214ED
:1030B30024900065E0FF12142430290FC2299000E8
:1030C300347405F090000074F0F02290004BE0FFA0
:1030D30012145390003D740AF0900000E004F022B3
:102F730090000EE0540F75F00AA4FFA3E0540F2F46
:102F8300F56B900011E0540F75F00AA4FDACF090BE
:102F93000010E0540F75F064A42DFFE5F03CFE90A3
:102FA3000012E0540F7C002FFFEC3EFEE56BC39450
:102FB300014019E56BD394145012C3EF9401EE94BE
:102FC300004009D3EF94FAEE9400400A12461F9092
:102FD300000074FAF02212476C90006CEEF0A3EF3D
:102FE300F090006CE475F001122E6BAFF0FEAD6B48
:102FF30012322C900011E0540F75F00AA4FF9000D8
:1030030010E0540F75F064A42FFF900012E0540FEA
:103013002FF56B90006CE0FEA3E0FFAD6B12322C3A
:0F3023007BFF7A0679F912462590000074FEF0C3
:01303200227B
:101F98007F0D122B18EF701A900011E0B43010A3C7
:101FA800E0B4300BA3E0B43006A3E0643060030271
:101FB8002091900015E0FF64306004EFB4350E9076
:101FC8000016E0540FD394054003022091900015A9
:101FD800E0FF64316004EFB4361190001AE0B420D9
:101FE80007900019E0B42003022091900015E0FF4B
:101FF80064326004EFB43711900019E0B420079000
:102008000018E0B42003022091900015E0FF64332B
:102018006004EFB43809900016E0B42002806A909A
:102028000015E0FF64346005EF64397066900016AF
:10203800E0540F75F00AA4FFA3E0540F2FF56B903E
:102048000019E0540F75F00AA4FDACF0900018E0F8
:10205800540F75F064A42DFFE5F03CFE90001AE0E3
:10206800540F7C002FFFEC3EFEE56BC39401401932
:10207800E56BD394145012C3EF9401EE9400400919
:10208800D3EF94FAEE9400400A12461F90000074B1
:10209800FAF02212476C90006CEEF0A3EFF090007B
:1020A8003D740AF0E4F56B900046E0FFE56BC39FD2
:1020B800502790006CE475F001122E6BAFF0FE9083
:1020C800003DE0FD04F074042DF582E43400F5834E
:1020D800E0FD12322C056B80CE7BFF7A0679F9126F
:0820E800462590000074FEF093
:0120F00022CD
:1033B400900048E0FF700330295B12145312476CED
:1033C40090006CEEF0A3EFF0E4F56B900046E0FFA4
:1033D400E56BC39F502C90006CE475F001122E6BCA
:1033E400AFF0FE1232698F6C7424256BF582E434DD
:1033F40000F583E56CF07E00123269121424056B2B
:1034040080C9302910C229E56B04900034F0900083
:103414000074F0F02290004BE0FF12145390003D32
:0B342400740AF0D226900000E004F0D3
:01342F00227A
:1037C800302365900001E0FF900035F0C223BF2A46
:1037D800079000007403F022900035E0FFB423083E
:1037E800900000E004F0803DEF547FFF1214249015
:1037F8000035E0547FFF90003DE0FE04F074042E95
:10380800F582E43400F583EFF0900046E02409FFE8
:10381800E433FE90003DE0D39FEE6480F874809816
:093828004006900000E004F022CB
:103F630030234B900001E0FF900035F0C223BF2ABD
:103F7300079000007403F022900035E0FFB4230B98
:103F8300900000E004F0E004F080101249EB500FC1
:103F9300900035E0900040F0900000E004F0227BB8
:0F3FA300FF7A0679D912462590000074FAF022B1
:10318F0020230302322B900001E0FF900035F0C2A4
:10319F0023BF2A079000007403F022900035E0FF50
:1031AF00B4230A900000E004F0E004F0221249EB8F
:1031BF00505B900040E0540F75F00AA4FF9000356B
:1031CF00E0540F2FF0E09008F293FF900035F012CB
:1031DF001424900035E0FF90003DE0FE04F07404ED
:1031EF002EF582E43400F583EFF0900046E02409D9
:1031FF00FFE433FE90003DE0D39FEE6480F87480CF
:10320F0098900000E0400304F02214F0227BFF7A34
:0D321F000679D912462590000074FAF022BD
:1047E600302009900077E0F55F121118302203E4BB
:1047F600F55F30210B301E05755F0A8003755F2853
:07480600900000E004F02225
:10383100E55F7063122C06900045E0122E8D386111
:103841006438666E38667838668238668C386B966E
:103851003870A03875AA387AB4387FBE0000388233
:10386100124935801C1246818017124A918012122A
:103871004A92800D124A938008124A948003124A98
:103881009530200D900076E0F55B900000E004F0AB
:08389100229000007401F022F6
:0E49FA00E55B700912111E9000007401F0229E
:103D1D0030200D900077E0F55F121118E55F70FC13
:103D2D00302107755F05E55F70FCE4F56B30210C04
:103D3D00124A531211BD124A791211BD30200C12C4
:103D4D004A5E1211BD124A791211BD056BE56BC3A6
:103D5D00940540D930200A900076E0F55BE55B7064
:073D6D00FC9000007401F05E
:013D7400222C
:014A8D002206
:014A8E002205
:014A8F002204
:10375B0030210A201E079000007401F02230200D4A
:10376B00900077E0F55F121118E55F70FC302107D0
:10377B00755F05E55F70FC302015124A5EE4F56B52
:10378B001211BD056BE56BC3940A40F4124A7930F4
:10379B002115124A53E4F56B1211BD056BE56BC392
:1037AB00940A40F4124A7930200A900076E0F55BD7
:0C37BB00E55B70FC1248C0E4900000F0D8
:0137C70022DF
:014A90002203
:10425D0030313B202338756064E53F547FFF900279
:10426D005D93900001F030260EE53F30E709EF90A9
:10427D00026D93900001F0D223C231900001E0B4A1
:0F428D002307900002E004F022E4900002F022E8
:10429C00302F3B202338756064E53D547FFF90023E
:1042AC005D93900001F030260EE53D30E709EF906C
:1042BC00026D93900001F0D223C22F900001E0B464
:0F42CC002307900002E004F022E4900002F022A9
:101B5E00202403021CCB302303021CCB900002E096
:101B6E00F56BE4F0756064124A87D223BF3007909C
:101B7E0000017430F022BF31079000017431F02261
:101B8E00BF32079000017432F022BF33079000017C
:101B9E007433F022BF34079000017434F022BF3545
:101BAE00079000017435F022BF360790000174369D
:101BBE00F022BF37079000017437F022BF3807902C
:101BCE0000017438F022BF39079000017439F022F9
:101BDE00BF23109000017423F0AF6B056B900002D1
:101BEE00EFF022BF2A07900001742AF022BF4107AE
:101BFE009000017441F022BF42079000017442F040
:101C0E0022BF43079000017443F022BF6407900087
:101C1E00017444F022202603C22322BF61079000E4
:101C2E00017461F022BF62079000017462F022BF5E
:101C3E0063079000017463F022BF64079000017483
:101C4E0064F022BF65079000017465F022BF66073D
:101C5E009000017466F022BF67079000017467F070
:101C6E0022BF68079000017468F022BF69079000D8
:101C7E00017469F022BF6A07900001746AF022BFF6
:101C8E006B07900001746BF022BF6C07900001741B
:101C9E006CF022BF6D07900001746DF022BF6E07CD
:101CAE00900001746EF022BF6F07900001746FF008
:0D1CBE0022BF70079000017470F022C22355
:011CCB0022F6
:0B4A23007F209000047420F0A3DFFC53
:014A2E002265
:0F49EB00EFC394304007EFD39439500122C32219
:1035990090000DE0FD6420602E90000CE0540F7542
:1035A900F00AA4FBAAF090000BE0540F75F064A494
:1035B9002BFFE5F03AFEED540F7C002FFFEC3E9017
:1035C9000068F0A3EF803190000CE0FD64209000CA
:1035D9000B601AE0540F75F00AA4FFED540F7C003C
:1035E9002FFEEC35F0900068F0A3CE800BE0540F6D
:1035F900FF900068E4F0A3EFF0E024FFF09000688A
:05360900E034FFF02297
:1039010090000AE0FD6420602B900009E0540F75DF
:10391100F00AA4FBAAF0900008E0540F75F064A42B
:103921002BFFE5F03AFEED540F7C002FFFEC3E90AB
:10393100006A802E900009E0FD6420900008601A62
:10394100E0540F75F00AA4FFED540F7C002FFEEC3C
:1039510035F090006AF0A3CEF022E0540FFF900002
:073961006AE4F0A3EFF0227D
:10489F00900006E0540F75F00AA4FFA3E0540F2F09
:1048AF00900036F0D394004006E09415500122C3D7
:0148BF0022D6
:103B5A00E4FFEF75F003A42409F582E43407F58342
:103B6A00E493FE900005E0FDEE6D703BEF75F00307
:103B7A00A4240AF582E43407F583E493FE90000650
:103B8A00E0FDEEB50521EF75F003A4240BF582E400
:103B9A003407F583E493FE900007E0FDEEB50507D0
:0C3BAA00900037EFF0D3220FBF33A7C309
:013BB60022EC
:103AFA00E4FF75F003EFA424A2F582E5F03407F59C
:103B0A0083E493FE900005E0FDEE6D703D75F003D1
:103B1A00EFA424A3F582E5F03407F583E493FE903D
:103B2A000006E0FDEEB5052275F003EFA424A4F526
:103B3A0082E5F03407F583E493FE900007E0FDEE9A
:0F3B4A00B50507900038EFF0D3220FBF70A4C36A
:013B59002249
:102B180074042FF582E43400F583E0FD64317069B4
:102B2800FE74052FF582E43400F583E0FCEE75F0C1
:102B380003A42409F582E43407F583E4936C704216
:102B480074062FF582E43400F583E0FCEE75F0039B
:102B5800A4240AF582E43407F583E493B5042374C6
:102B6800072FF582E43400F583E0FCEE75F003A44A
:102B7800240BF582E43407F583E493B50404EE04EA
:102B8800FF220EBE339B7F0022ED6432706DFE740F
:102B9800052FF582E43400F583E0FD75F003EEA41B
:102BA80024A2F582E5F03407F583E4936D7045744B
:102BB800062FF582E43400F583E0FD75F003EEA4FA
:102BC80024A3F582E5F03407F583E493B50525746D
:102BD800072FF582E43400F583E0FD75F003EEA4D9
:102BE80024A4F582E5F03407F583E493B50505EEF2
:0D2BF8002434FF220EBE70977F00227F0064
:012C050022AC
:1032B200EFC3943390006350397431F0EF75F0032B
:1032C200A42409F582E43407F583E493900064F0C2
:1032D200EF75F003A4240AF582E43407F583E4933E
:1032E200900065F0EF75F003A4240BF582E4340737
:1032F200803A7432F075F003EFA42409F582E5F008
:103302003407F583E493900064F075F003EFA4248E
:103312000AF582E5F03407F583E493900065F075D1
:10332200F003EFA4240BF582E5F03407F583E49370
:05333200900066F0228E
:10497800900006E0540F75F00AA4FFA3E0540F2F2F
:05498800900039F0224F
:10498D00900006E0540F75F00AA4FFA3E0540F2F1A
:05499D0090003AF02239
:1049A200900006E0540F75F00AA4FFA3E0540F2F05
:0549B20090003BF02223
:06461F007BFF7A067949D9
:064625008B6C8A6D896EAA
:10462B007F01121453E4F56FAB6CAA6DA96E856F05
:10463B0082758300122DD7FF121424056FE56FC30B
:04464B00941040E4A3
:01464F002248
:064650007BFF7A06799958
:064656008B6C8A6D896E79
:10465C007F11121453E4F56FAB6CAA6DA96E856FC4
:10466C0082758300122DD7FF121424056FE56FC3DA
:04467C00941040E472
:014680002217
:10476C00900050E0FF7E00900051E0FCA3E0FD12B1
:10477C002E0490004FE02FFF90004EE03EFE900084
:0A478C0047E07C002FFFEC3EFE2208
:1049B700900049E075F010A424DDF9740935F0FA88
:0549C7007BFF024656D3
:034A87007F032288
:1048FF00E4F56BAF6B7E00E56B900B3D93FD1232D1
:0A490F002C056BE56BC3941040E922
:01491900227B
:10443E00E4F56BE4F56CE56B75F017A42464FFE40A
:10444E0035F0FE7C00EF256CFFEC3EFEE56C900B2C
:10445E006193FD12322C056CE56CC3941740D705A1
:08446E006BE56BC3946440CBC5
:014476002223
:10480D00E4F56BAF6B7E00123269746E256BF58229
:10481D00E43400F583EFF0056BE56BC3941040E3D2
:06482D0090006EE0F52092
:014833002262
:10493500302008900024E0FF124A3B302108900007
:0749450024E0FF124A2F22BB
:10468100E4F56B900034E0FFE56BC39F5021742487
:10469100256BF582E43400F583E0F56C302004FFEE
:0F46A100124A3B302105AF6C124A2F056B80D4B3
:0146B00022E7
:014A91002202
:014A92002201
:014A93002200
:014A940022FF
:014A950022FE
:0C4A2F00124A691211BD124A800211BD2A
:0C4A3B00124A711211BD124A800211BD16
:102C0600E4F56BF56CF56D900069E02401FF90002A
:102C160068E03400FEC3EF940AEE94005005A3E08A
:102C260004F56DD3EF9463EE9400404C900069E098
:102C36002401FB900068E03400FA7C007D64AF0359
:102C4600FE122E168F6BEF75F064A4FFC3EB9FFF89
:102C5600EA95F0FE7C007D0A122E168F6CA3E00426
:102C6600FFE56B75F064A4FEC3EF9EFFE56C75F09F
:102C76000AA4FEC3EF9EF56D900069E02401FF9063
:102C86000068E03400FED3EF9409EE940040197C0E
:102C9600007D0A122E168F6CA3E004FFE56C75F01A
:102CA6000AA4FEC3EF9EF56D7430256BF56B743088
:102CB600256CF56C7430256DF56D302014AF6B12F4
:102CC6004A3BAF6C124A3BAF6D124A3B7F2A124A0F
:102CD6003B302114AF6B124A2FAF6C124A2FAF6DE7
:082CE600124A2F7F2A124A2F27
:012CEE0022C3
:1040D5002A2A3132333435362A2A2A2A31323334E0
:1040E50035302A2A44313233343536373839302A97
:1040F50023414243202056455253494F4E20312EED
:10410500312020202043442D322043415220504C61
:0441150055532020BE
:1030E300302A28C22AE53F540F9040E99390009379
:1030F300F0301D03123A32754C32900084E004F034
:1031030030011412454F12438F800CE54C70089028
:10311300007FF0900090F0302B3DC22BE53D540F23
:103123009040E993900092F01239CE754D329000A1
:1031330084E004F0301E03200006201E0630020344
:10314300124354301E03200003201E0312451A208D
:103153001E111245EC800CE54D7008900080F09034
:10316300008FF03025193003221239CE754E3212FA
:103173004A8A900083EFF0C2251243CA024584E5D0
:0C3183004E7008900081F0900091F02246
:10451A00900080E0FF04F0EF9040D593FF90009266
:10452A00E0FEEF6E6011EEB42A089000807401F08C
:10453A008005E4900080F0900080E0B40A06E4F080
:05454A00D221D22C2259
:10454F0090007FE0FF04F0EF9040D593FF90009331
:10455F00E0FEEF6E6011EEB42A0890007F7401F058
:10456F008005E490007FF090007FE0B40A06E4F04D
:05457F00D220D22C2225
:10458400900081E0FF04F0EF9040D593FF9000830A
:10459400E0FEEF6E6011EEB42A089000817401F021
:1045A4008005E4900081F0900081E0B40A06E4F014
:0545B400D222D22C22EE
:1043540090008FE0FF04F074862FF582E43400F5BA
:1043640083E0FF900092E0FEEF6E6011EEB423084C
:1043740090008F7401F08005E490008FF090008F1E
:0B438400E0B40906E4F0D221D21F22B1
:10438F00900090E0FF04F074862FF582E43400F57E
:10439F0083E0FF900093E0FEEF6E6011EEB4230810
:1043AF009000907401F08005E4900090F0900090E0
:0B43BF00E0B40906E4F0D220D21F2277
:1043CA00900091E0FF04F074862FF582E43400F542
:1043DA0083E0FF900083E0FEEF6E6011EEB42308E5
:1043EA009000917401F08005E4900091F0900091A2
:0B43FA00E0B40906E4F0D222D21F223A
:1045EC00900082E0FF04F0EF9040DF93FF90009288
:1045FC00E0FEEF6E6011EEB42A089000827401F0B8
:10460C008005E4900082F0900082E0B40A04E4F0AB
:03461C00D22D227A
:10473F009000867423F0A3F0E4FF746F2FF582E4EA
:10474F003400F583E0FE74882FF582E43400F5839E
:0C475F00EEF00FBF06E490008E7423F013
:01476B00222B
:1042DB0012138112146D12147CE4900084F07BFF96
:1042EB007A4179091246257BFF7A4079F9124656B5
:1042FB00752F147F10900053E4F0A3DFFC7F10E5C3
:0E430B002F70FC12146D12147C7F01021453EB
:1048C00012138112146D12147CE4900084F07F1096
:1048D000900053E4F0A3DFFC12146D7F0102145327
:1039CE00900084E0FED3940F5012900092E0FF74AA
:1039DE00532EF582E43400F583EF80437F011214F9
:1039EE0053E4F56B7454256BF582E43400F583E0F3
:1039FE00FF7453256BF582E43400F583EFF07453B6
:103A0E00256BF582E43400F583E0FF121424056B78
:103A1E00E56BC3940F40CD900092E0FF900062F0F2
:033A2E001214244B
:013A31002272
:103A3200900084E0FED3940F5012900093E0FF7444
:103A4200532EF582E43400F583EF80437F01121494
:103A520053E4F56B7454256BF582E43400F583E08E
:103A6200FF7453256BF582E43400F583EFF0745351
:103A7200256BF582E43400F583E0FF121424056B14
:103A8200E56BC3940F40CD900093E0FF900062F08D
:033A9200121424E7
:013A9500220E
:034A8A007F012287
:1019C4007549001219DF50FB22754900121A68503C
:1019D400FB22754900121A1F50FB22758400E54949
:1019E40075F003A49019EC73021A84021A93021A74
:1019F400B1021A9A021ABD021AC4021ACC021A932C
:101A0400021ADA021A9A021AEA021AF3021A84026F
:101A14001A93021B01021A9A021B0D758400E549F0
:101A240075F003A4901A2C73021A84021A93021AF2
:101A3400B1021A9A021ABD021AC4021A84021A9333
:101A4400021AB1021A9A021ABD021AC4021ABD027B
:101A54001AC4021ACC021A93021B0F021A9A021A0F
:101A6400EA021B0D758400E54975F003A4901A750C
:101A740073021A84021A93021B01021A9A021B0DA2
:101A8400C2FA121B1F121B1F759B000549C322308B
:101A9400F9020549C32230F912E59A20E7FB121B2B
:101AA4001FD2FA121B1F121B1F0549C322C2FA12AE
:101AB4001B1F759B040549C322752E1E0549C322AD
:101AC400E52E70020549C322C2FA121B1F121B40E5
:101AD400F59B0549C322C2FA121B1F121B4F440770
:101AE400F59B0549C322121B31F52F0549C3227505
:101AF400840F30DE04E52F70020549C322C2FA12B6
:101B04001B1F759B080549C322D322C2FA121B1F4F
:091B1400121B4F4405F59B054925
:101B1D00C3220000000000000000000000000000D3
:101B2D0000000022901B38E54A93225A5A5A5A5AFD
:101B3D00FAFAFA901B47E54A932200B45AE12D8731
:101B4D007ADB901B56E54A932200000000000080CE
:011B5D008007
:10360E0075840F1200A412480D12473F1242DBE4DC
:10361E0090007EF01246B11230E3123A96302D052C
:10362E00123430C22D302C2FC22C7F0C12149A1251
:10363E0048FF12443E12480D12473FE490007EF0C0
:10364E00C220C221C222F56A1211BD056AE56AC303
:10365E00941E40F41248C0301FBA1245B912480DDC
:10366E0012473FE490007EF0C220C221C22280A405
:103A9600900041E07014121161400F1211307563ED
:103AA60064124A53900041E004F0900041E0B401F2
:103AB60010E563703E124A7975623C900041E0045D
:103AC600F0900041E06402701E121173500512114D
:103AD6006D4007E5627010201F0D12113875636482
:103AE600900041E004F022900041E0B40305E56354
:043AF6007001F02249
:102A100009920A9E0BC70D100E7D101211D213C51C
:102A200015ED185208D0094E09D40A600AF40B912A
:102A30000C360CE50D9D0E600F2D100610EB11DD10
:102A400012DC13EA15071633177118C01D2107B1E0
:102A500007E808200859196E1A211ADA1B971C5A20
:102A60000894090E09900A190AA90B410BE30C8C72
:102A70000D3F0DFD0EC50F9810771162125B1362AA
:102A80001477159B16D018161DEF1EC21F9B2079B8
:102A9000215F224A233B24342533263912330FCDBC
:102AA00014331566169A17CD19000E9A1366110085
:102AB00011661033150016331766189A19CD0DCD0F
:102AC0000F00129A11CD1300149A15CD1700183368
:102AD00019660E330F66109A191823A01296203D1E
:102AE000129623A0129627631488203D148823A0F1
:102AF0001488276316B8203D16B823A016B827639C
:102B00001918203D1918276312962B8C14882B8CCA
:082B100016B82B8C19182B8C50
:0B4A530075081575095ED233D20B22E6
:0B4A5E0075081575095ED233D21322D3
:074A7900C233C20BC213227D
:084A6900121E37D234D20C22D8
:084A7100121E37D234D21422C8
:091E3700E4F512F513F514F5159C
:101E4000EF122E8D1F3B231F2A2A1E78301E8A3147
:101E50001E9C321EAE331EC0341ED2351EE4361E0A
:101E6000F6371F08381F19391F4C411F5D421F6E7E
:101E7000431F7F4400001F97902AD8E493F50D7408
:101E80000193F50E902ADA021F8E902ADCE493F576
:101E90000D740193F50E902ADE021F8E902AE0E465
:101EA00093F50D740193F50E902AE2021F8E902A8D
:101EB000E4E493F50D740193F50E902AE6021F8E6B
:101EC000902AE8E493F50D740193F50E902AEA0246
:101ED0001F8E902AECE493F50D740193F50E902A71
:101EE000EE021F8E902AF0E493F50D740193F50E27
:101EF000902AF2021F8E902AF4E493F50D74019358
:101F0000F50E902AF6021F8E902AF8E493F50D74D0
:101F10000193F50E902AFA8075902AFCE493F50D52
:101F2000740193F50E902AFE8064902B00E493F5E3
:101F30000D740193F50E902B028053902B04E493C3
:101F4000F50D740193F50E902B068042902B08E45A
:101F500093F50D740193F50E902B0A8031902B0CA4
:101F6000E493F50D740193F50E902B0E8020902BC9
:101F700010E493F50D740193F50E902B12800F90E1
:101F80002B14E493F50D740193F50E902B16E49346
:081F9000F50F740193F5102216
:074A8000C234C214C20C2273
:1049CC0044313233343536373839302A2341424377
:1046B100124A1612479690007EE01460131460139C
:1046C1001460131460131460132405701202494C12
:1046D100022CEF0246E102485902496212491A22AC
:10494C00E4F564E56490007E700804F0E490008562
:06495C00F0227414F022A9
:102CEF0090004EE4F0A37464F09000507417F0E479
:102CFF00900051F0A3F0E4900047F012476C1232AD
:102D0F0069900047E0FE900051E0FCA3E09000FACC
:102D1F0075F006122E81EC75F006A42583F583E578
:102D2F00822EF582E43583F583EFF0900047E004BF
:102D3F00F0E0C3940640C49000477406F012476C4D
:102D4F00123269AD07900052E0C4F8540FC868FF03
:102D5F00900051E0C454F048FE744C2FF582740378
:102D6F003EF583C083C082900047E0D082D0832598
:102D7F0082F582E43583F583EDF0900047E004F0AF
:102D8F00E0C3941640B79000477416F012476C12C8
:102D9F003269900052E02492F582E43409F583EF12
:102DAF00F0900052E004F07006900051E004F0C380
:102DBF00900052E09464900051E094005003022D73
:082DCF000590007EE004F022F3
:1046E100744A4408602990007DE0F57012147C7FC3
:1046F10001121453E4900085F09000537420F0A34C
:10470100F0A3F0A3F0A3F0A3F090007EE004F02268
:10485900E570700D90007CE0F57190007EE004F049
:1048690022124A08500C12487C12389990007DE0B7
:03487900F57022B5
:10496200120B7812447712483490007CE0F5719073
:06497200007EE004F022CB
:10491A0090007CE06006E57170028005124A08503A
:0B492A00091248C090007E7402F022C9
:10479600301C250569E569AE687002056814249623
:1047A600F58274003EF583E53FF0C21CE56964645A
:0947B60045687004F568F56922FC
:0E4A0800E569B56707E568B56602C322D322EB
:10487C000567E567AE6670020566142496F58274CA
:10488C00003EF583E0FFE567646445667004F566F9
:02489C00F567BE
:01489E0022F7
:10389900EF540F9049CC93F56B900085E0D3940FCA
:1038A9005010E0FF04F074532FF582E43400F583DF
:1038B900803E7F01121453E4F56C7454256CF58233
:1038C900E43400F583E0FF7453256CF582E4340099
:1038D900F583EFF07453256CF582E43400F583E049
:1038E900FF121424056CE56CC3940F40CD9000625F
:0738F900E56BF0FF1214243F
:0139000022A4
:100B7800C23AE4F56B75F006E56BA424FAF582E554
:100B8800F03400F583E0FF1249EB4003020C4E7588
:100B9800F006E56BA424FAF582E5F03400F583E06D
:100BA800FF900053E0FEEF6E6003020E8E75F006B4
:100BB800E56BA424FBF582E5F03400F583E0FF90B3
:100BC8000054E0FEEF6E6003020E8E75F006E56BD2
:100BD800A424FCF582E5F03400F583E0FF9000558D
:100BE800E0FEEF6E6003020E8E75F006E56BA4243E
:100BF800FDF582E5F03400F583E0FF900056E0FE55
:100C0800EF6E6003020E8E75F006E56BA424FEF508
:100C180082E5F03400F583E0FF900057E0FEEF6EC8
:100C28006003020E8E75F006E56BA424FFF582E5DD
:100C3800F03400F583E0FF900058E0FEEF6E6003AB
:100C4800020E8E020E8875F006E56BA424FBF58271
:100C5800E5F03400F583E0FF1249EB4003020D0193
:100C680075F006E56BA424FBF582E5F03400F58306
:100C7800E0FF900054E0FEEF6E6003020E8E75F008
:100C880006E56BA424FCF582E5F03400F583E0FF6B
:100C9800900055E0FEEF6E6003020E8E75F006E5DB
:100CA8006BA424FDF582E5F03400F583E0FF9000A5
:100CB80056E0FEEF6E6003020E8E75F006E56BA43B
:100CC80024FEF582E5F03400F583E0FF900057E05C
:100CD800FEEF6E6003020E8E75F006E56BA424FF2E
:100CE800F582E5F03400F583E0FF900058E0FEEF70
:100CF8006E6003020E8E020E8875F006E56BA42462
:100D0800FCF582E5F03400F583E0FF1249EB507BF7
:100D180075F006E56BA424FCF582E5F03400F58354
:100D2800E0FF900055E0FEEF6E6003020E8E75F056
:100D380006E56BA424FDF582E5F03400F583E0FFB9
:100D4800900056E0FEEF6E6003020E8E75F006E529
:100D58006BA424FEF582E5F03400F583E0FF9000F3
:100D680057E0FEEF6E6003020E8E75F006E56BA489
:100D780024FFF582E5F03400F583E0FF900058E0A9
:100D8800FEEF6E6003020E8E020E8875F006E56BAC
:100D9800A424FDF582E5F03400F583E0FF1249EB69
:100DA800505D75F006E56BA424FDF582E5F034008E
:100DB800F583E0FF900056E0FEEF6E6003020E8EB2
:100DC80075F006E56BA424FEF582E5F03400F583A2
:100DD800E0FF900057E0FEEF6E6003020E8E75F0A4
:100DE80006E56BA424FFF582E5F03400F583E0FF07
:100DF800900058E0FEEF6E6003020E8E020E8875BA
:100E0800F006E56BA424FEF582E5F03400F583E0F6
:100E1800FF1249EB503875F006E56BA424FEF58205
:100E2800E5F03400F583E0FF900057E0FEEF6E70C8
:100E38005575F006E56BA424FFF582E5F03400F55E
:100E480083E0FF900058E0FEEF6E703A803275F054
:100E580006E56BA424FFF582E5F03400F583E0FF96
:100E68001249EB502175F006E56BA424FFF582E5E5
:100E7800F03400F583E0FF900058E0FEEFB5060679
:100E8800D23A856B6522056BE56BC3946450030207
:020E98000B7DD0
:010E9A002235
:10447700203A0302147C7F11121453E4F56B75F094
:1044870010E565A42452F582E5F03403F583E5824F
:10449700256BF582E43583F583E0FF121424056B61
:0744A700E56BC3941040D740
:0144AE0022EB
:10483400303A1374922565F582E43409F583E06017
:104844001390007B800630040B90007AE0F572D25E
:054854003B12112422BB
:0D4A1600303B09E572700512112AC23B22E7
:03000000024A476A
:0C4A4700787FE4F6D8FD7581A202360EDF
:102DD700BB010CE58229F582E5833AF583E02250B1
:102DE70006E92582F8E622BBFE06E92582F8E222FB
:0D2DF700E58229F582E5833AF583E4932215
:102E0400EF8DF0A4A8F0CF8CF0A428CE8DF0A42EE2
:022E1400FE229C
:102E1600BC000BBE0029EF8DF084FFADF022E4CCA0
:102E2600F875F008EF2FFFEE33FEEC33FCEE9DEC69
:102E3600984005FCEE9DFE0FD5F0E9E4CEFD22EDAF
:102E4600F8F5F0EE8420D21CFEADF075F008EF2FF9
:102E5600FFED33FD4007985006D5F0F222C398FDEA
:052E66000FD5F0EA2287
:102E6B00A3F8E0C5F025F0F0E5821582700215831A
:062E7B00E0C838F0E82277
:0C2E8100A42582F582E5F03583F583225C
:102E8D00D083D082F8E4937012740193700DA3A3D4
:102E9D0093F8740193F5828883E4737402936860E8
:062EAD00EFA3A3A380DFE8
:00000001FF
